:100000001DC0189518951895189518950BC1189539
:100010001895189518954156525F53303035205633
:10002000312E30302031342E30372E3230303420E3
:10003000482E205072696E7A6C6572000FED0DBF0C
:1000400000E007BB0FE108BB0EE001BB08E002BB0C
:10005000479A05B70F7E006205BFF7D0E0E7F1E0F1
:1000600001D1F0E0E6E5FED07894939804E10093A6
:100070006C000ED153FDF9CF00916C00002329F0E4
:100080000A9500936C008895F4CF939A08EC00933E
:100090006C00FED053FDE9CF00916C0000230023DB
:1000A00021F30A9500936C008895F3CF5527F0E073
:1000B000E7E8F0936A00E09369000EE200936B00BA
:1000C00002BF02E003BF08B7026008BF09B70260C1
:1000D00009BFDED050FDFDCF00271127B09B016086
:1000E000B19B0260B29B0460B39B0860B49B00614B
:1000F0000113586053FFEDCF011301C0577F006A11
:10010000101B00936500109366005160E2CF20E061
:1001100023BF2EE922BF25E023BF8FD020E023BFDD
:100120002EE222BF22E023BF88D050FFF0CF5260E2
:100130002AE020936000929A20916000222329F007
:100140002A95209360005B7F02C05D7F546075D06C
:1001500052FF01C0929871D092986FD051FDEBCFB1
:10016000209165002093670020916600209368002D
:100170005E7F22E02093610020E02093630027E669
:1001800020936200EF93FF93E0916200F09163008F
:100190002191E0936200F0936300FF91EF9120932F
:1001A000640028E020936000929A2091600022234E
:1001B00071F02A95209360002091640020FF02C016
:1001C000546001C05B7F2695209364001CC054607E
:1001D000209161002A9520936100222309F413C025
:1001E000EF93FF93E0916200F09163002191F0930F
:1001F0006300E0936200FF91EF912093640028E098
:100200002093600000C019D052FF01C0929815D011
:10021000929813D020916100222309F0C5CF50FDA0
:1002200086CF75CF0FB620916B0022BF2091690059
:100230002F9320916A002F9308952F9120936A00A5
:100240002F91209369000FBE189500E000936D0078
:1002500001E000936E0001E700936F0000E000935F
:100260007000089500916E0015E0011781F0102FC5
:10027000039500936E00EF93FF93110FE1E7E10FF9
:10028000F0E01127F11F0F9101830F910083089572
:10029000E0916F00F09170000F9101830F91008346
:1002A00000916D0010916E000395011709F400276D
:1002B00000936D00E1E7F0E0000FE00F0027F01F72
:1002C000E0936F00F093700000810F9301810F9312
:1002D00008954D4F4E4930312056312E30300000B8
:1002E00048E14AB949E149B9909A4CB1D1DF26D0E9
:1002F000053AE9F723D000937B0020D000937C00DF
:100300001DD000937D001AD0013019F4E9E6F1E028
:100310003EC0023019F4EBE0F0E039C0033009F4DC
:100320005DC0043009F479C0053009F48AC0063094
:1003300009F49DC0073009F4A1C0D9CF5F990FC05F
:100340000F9100937F000F9100937E00A1DF5F9BD0
:10035000FDCF00917E000F9300917F000F930CB1B1
:100360005C99ECCF0895402F5D990FC00F910093D9
:100370007F000F9100937E008BDF5D9BFDCF00918E
:100380007E000F9300917F000F934CB90895EE0FFC
:10039000FF1FF0937B00E0937C0000917D00002321
:1003A000E1F00A9500937D00F0917B00E0917C00E4
:1003B000C895002041F03196F0937B00E0937C00DB
:1003C000002DD1DFEACF00E2CEDF00917D000023D7
:1003D00021F00A9500937D00F6CF89CFF0917B0044
:1003E000E0917C00EE0FFF1FF0937B00E0937C0018
:1003F00000917D00002381F00A9500937D00F0912B
:100400007B00E0917C00C8953196F0937B00E093EF
:100410007C00002DA8DFECCF6ACF00917D00002387
:1004200079F00A9500937D00F0917B00E0917C00CB
:1004300000813196F0937B00E0937C0094DFEDCF58
:1004400056CFE199FECF00917D00002379F00A9507
:1004500000937D00E0917C00EEBBE09A0DB33196F5
:10046000F0937B00E0937C007EDFEDCF40CF66DF32
:10047000F0917B00E0917C00008339CFE199FECFC1
:100480005DDFE0917C00EEBB0DBBE29AE19A2FCFDD
:00000001FF
